:020000040000FA
:1000000008200020150200001D0200001F02000051
:100010002102000023020000250200000000000071
:1000200000000000000000000000000027020000A7
:1000300029020000000000002B0200002D02000039
:100040002F0200002F0200002F0200002F020000EC
:100050002F0200002F0200002F0200002F020000DC
:100060002F0200002F0200002F0200002F020000CC
:100070002F0200002F0200002F0200002F020000BC
:100080002F0200002F0200002F0200002F020000AC
:100090002F0200002F0200002F0200002F0200009C
:1000A0002F0200002F0200002F0200002F0200008C
:1000B0002F0200002F0200000000000000000000DE
:1000C0002F0200002F0200002F0200002F0200006C
:1000D0002F0200002F0200002F020000000000008D
:1000E0000000000000000000000000000000000010
:1000F0000000000000000000000000000000000000
:1001000000000000000000000000000000000000EF
:1001100000000000000000000000000000000000DF
:1001200000000000000000000000000000000000CF
:1001300000000000000000000000000000000000BF
:1001400000000000000000000000000000000000AF
:10015000000000000000000000000000000000009F
:10016000000000000000000000000000000000008F
:10017000000000000000000000000000000000007F
:10018000000000000000000000000000000000006F
:10019000000000000000000000000000000000005F
:1001A000000000000000000000000000000000004F
:1001B000000000000000000000000000000000003F
:1001C000000000000000000000000000000000002F
:1001D000000000000000000000000000000000001F
:1001E000000000000000000000000000000000000F
:1001F00000000000000000000000000000000000FF
:10020000DFF80CD000F018F8004800473506000071
:10021000082000200648804706480047FEE7FEE722
:10022000FEE7FEE7FEE7FEE7FEE7FEE7FEE7FEE7A6
:100230005D02000001020000064C074D06E0E06888
:1002400040F0010394E8070098471034AC42F6D31D
:10025000FFF7DAFFB0060000D0060000F0B5B548A1
:100260000023021D0178101D01254FF0805406293E
:100270000BD11678360708D10678C6F30316032E7D
:1002800006D0042E04D0052E02D0062907D00EE099
:10029000B4F82463A84FC6F304263E6002E0167843
:1002A000360704D10678C6F30316032E02D00629BA
:1002B00004D00FE0A24FA14E7E670EE016783607FD
:1002C00008D10678C6F30316032E06D0042E04D0F8
:1002D000052E02D0062907D00EE0D4F84462994FCB
:1002E000C6F342363E6002E01678360704D106783F
:1002F000C6F30316032E02D0062906D011E0924E53
:10030000376827F0807737600EE01678360708D117
:100310000678C6F30316032E06D0042E04D0052E4D
:1003200002D006290AD011E04FF08046C6F80C3101
:10033000C6F81031834E361F336002E01678360758
:1003400004D10678C6F30316032E02D0062905D081
:100350000CE07C4F032664373E600AE016783607CF
:1003600004D10678C6F30316032E02D006290DD059
:1003700014E0764F05263E60744E78363560734E35
:10038000083633603F263F1D3E6002E01678360790
:1003900004D10678C6F30316052E02D0062957D0DD
:1003A00062E06B4E36686B4F3E60694E361D3668B4
:1003B0003F1D3E60664E083636683F1D3E60644E07
:1003C0000C3636683F1D3E60614E103636683F1D64
:1003D0003E605F4E143636683F1D3E605C4E1836F8
:1003E00036685C4F20373E60594E1C3636683F1DDC
:1003F0003E60574E203636683F1D3E60544E2436D0
:1004000036683F1D3E60524E283636683F1D3E60BE
:100410004F4E2C3636683F1D3E604D4E30363668A6
:100420004C4F40373E604A4E343636683F1D3E6082
:10043000474E383636683F1D3E60454E3C3636687E
:100440003F1D3E60424E403636683F1D3E6002E032
:100450001678360708D10678C6F30316032E06D0A1
:10046000042E04D0052E02D0062907D019E0D4F8B6
:100470005812394A01F04F01116002E01178090762
:100480000FD10078C0F30310032803D0042801D053
:10049000052806D131480168C90702D06FF0010173
:1004A0000160D4F83001062808D1D4F834010628B8
:1004B00004D12B48016841F48061016022487438FE
:1004C000016841F470010160BFF34F8FBFF36F8F7C
:1004D0004FF01021D1F80002002803DBD1F804020C
:1004E000002822DA1F4A15601F480468002CFCD03F
:1004F0001524C1F800420568002DFCD0C1F8044263
:1005000001680029FCD0136001680029FCD0BFF30A
:100510004F8F0D48F0380168144A01F4E06111432F
:100520000160BFF34F8F00BFFDE71249104808601C
:10053000F0BD0000E00F00F0403501400DF0ADBA15
:1005400000C007403C050040FCED00E010560040B4
:100550000404001020C50040E40E004000040040E8
:100560003C17004004E5014000E401400400FA05A6
:100570000090D0030000002002E008C8121F08C14C
:10058000002AFAD170477047002001E001C1121F14
:10059000002AFBD1704700002DE9FC410646C00748
:1005A0004FF000050ED0104F00240122385D009559
:1005B00000231146019500F055F8641C042CF4D377
:1005C00000F02EF8B0070DD5074E0024361D00228E
:1005D000305D032300951146019500F043F8641C3B
:1005E000042CF4D3BDE8FC81A606000007490B5C8F
:1005F0004FF0A041D1F804250120984020EA0203E1
:10060000C1F808351040C1F80C057047A606000077
:100610000249085C012100F037B80000A60600007E
:1006200010B500242046FFF7F3FF641C042CF9D317
:1006300010BD00000120FFF7AFFF094C4FF4FA781E
:100640004FF47A4700263046FFF7D0FF4546611C3D
:10065000384688476D1EFAD1761C042EF3DBF1E78D
:10066000A006000070B541EA4201DDE904564FF0F2
:10067000A04441EA830141EA052104EB800041EAFC
:100680000641C0F8001770BD01224FF0A043824020
:1006900011B1C3F808257047C3F80C257047000056
:1006A0000338FDD87047111213140D0E0F100000FF
:1006B000D0060000000000200400000078050000C3
:1006C000D40600000400002004200000880500007B
:0406D0000090D003C3
:0400000500000201F4
:00000001FF
